:020000040000FA
:020000000528D1
:08000800090000308B008501A6
:1000100086018316033085000030860083124E204F
:10002000051C1E2085181928083091008615061118
:100030001D28043091008611061510285F20051830
:1000400008004B2005150830110603192928003037
:100050002A2809309000100E11048600083011067D
:10006000031D3828FF30100603193F2890033D2850
:100070000930100603193F28900A69202B2806151D
:10008000861506144E2069206920692069206920A0
:1000900006100511080032308E00532864308E009F
:1000A000532896308E0086145A2086105A208E0BC4
:1000B0005328080002308C0000308F00732806306F
:1000C0008C0000308F00732801308C0001308F00CD
:1000D000732806308E0001308F00FF308C000F181F
:1000E0008E0B73280800FF308D008D0B75288C0B4C
:0800F00073280F186D280800A9
:02400E00F93F78
:00000001FF
